:1000000029C043C042C041C040C03FC03EC03DC007
:100010003CC03BC03AC039C038C037C036C035C01C
:1000200034C033C032C0084AD73B3BCE016E84BCDB
:10003000BFFDC12F3D6C74319ABD56833DDA3D0042
:10004000C77F11BED9E4BB4C3E916BAAAABE00008B
:1000500000803F0011241FBECFE5D4E0DEBFCDBF3E
:1000600011E0A0E6B0E0ECE6F9E102C005900D92E7
:10007000A637B107D9F711E0A6E7B1E001C01D929C
:10008000A639B107E1F720D16FCCBACFA59A8AE0A3
:10009000982F9A95F1F7A49A982F9A95F1F7A59829
:1000A000982F9A95F1F7A4988A95F1F71092760116
:1000B0009C9905C0809176018F5F809376019D9910
:1000C00005C0809176018F5F809376018AE0982F3A
:1000D0009A95F1F7982F9A95F1F7982F9A95F1F74D
:1000E0008A95F1F70895A498A598AC98AD98CEDFBD
:1000F000CDDF0895A49A8AE0982F9A95F1F7A59AF2
:100100008A95F1F70895A4988AE0982F9A95F1F7C7
:10011000A598982F9A95F1F7A49A982F9A95F1F7A8
:10012000A59A8A95F1F7089520E04AE087FD02C07C
:10013000A49A01C0A4983AE0942F9A95F1F7A59853
:10014000942F9A95F1F7A59A2F5F283011F0880F18
:10015000EDCFA498832F8A95F1F7A598832F8A95E0
:10016000F1F783B3A59A90E024E0969587952A95B8
:10017000E1F781700895A49820E030E04AE0330F61
:10018000A598942F9A95F1F79C993160A59A942F90
:100190009A95F1F72F5F283091F7882311F4A49AEC
:1001A00001C0A4988AE0982F9A95F1F7A598982F06
:1001B0009A95F1F7A59A8A95F1F7A498832F089557
:1001C0000F931F93182F062F95DF86EAADDF812F3F
:1001D000ABDF802FA9DF5ADF1F910F9108958DE2C9
:1001E00068E2EEDF81E368E0EBDF88E360E0E8DF10
:1001F000089580DF86EA98DF82E396DF47DF7ADFC3
:1002000087EA92DF80E0B7DF80937C0180E0B3DF94
:100210008093900180E0AFDF80938F0180E0ABDFBF
:100220008093770180E0A7DF8093910181E0A3DFD5
:1002300080937E012BDF9091900180E020917C01E2
:10024000820F911DAA2797FDA095BA2F80938B014D
:1002500090938C01A0938D01B0938E0190917701C2
:1002600080E020918F01820F911DAA2797FDA09514
:10027000BA2F8093780190937901A0937A01B0937B
:100280007B0190917E0180E020919101820F911D70
:10029000AA2797FDA095BA2F80938301909384019C
:1002A000A0938501B0938601089524DF86EA3CDFA0
:1002B00080E03ADFEBDE1EDF87EA36DF81E05BDFDE
:1002C00080937D01E3DE08952F923F924F925F92DB
:1002D0006F927F928F929F92AF92BF92CF92DF9256
:1002E000EF92FF920F931F93DF93CF93CDB7DEB7BB
:1002F0002C970FB6F894DEBF0FBECDBF8FE387BB40
:1003000018BA31D3F0DE6BDF81E021D380EA9FE0C1
:100310000197F1F7CADF80917D01853E29F484E8D9
:1003200016D380E690E04FD364DF80918B019091EB
:100330008C01A0918D01B0918E0189879A87AB873E
:10034000BC87209078013090790140907A015090DC
:100350007B01C201B101AAD69B01AC010BD53B01C7
:100360004C018091830190918401A0918501B0910D
:1003700086018D839E83AF83B887BC01CD0196D65D
:100380009B01AC01F7D45B016C01C401B301A60170
:100390009501C9D4F3D97B018C0169857A858B8558
:1003A0009C8590958095709561957F4F8F4F9F4F5D
:1003B0007DD6A8019701D3D517D924E13EE245E6C1
:1003C00052E4D8D4CDD669837A838B839C8360939F
:1003D00092017093930180939401909395016985A4
:1003E0007A858B859C8562D69B01AC01C3D47B0149
:1003F0008C01C801B701A601950195D4BFD95B0155
:100400006C015094409430942094211C311C411C68
:10041000511CC201B1014AD6A6019501A0D5E4D86C
:1004200024E13EE245E652E4A5D49AD65B016C0194
:1004300060937F017093800180938101909382018A
:10044000C801B701A40193016ED498D97B018C0136
:100450006D817E818F81988590958095709561954D
:100460007F4F8F4F9F4F22D6A801970178D5BCD8D8
:1004700024E13EE245E652E47DD472D660938701E2
:10048000709388018093890190938A0189819A8170
:10049000AB81BC81865A9F4FAF4FBF4F86349105C9
:1004A000A105B10510F4C09AC19889819A81AB81E8
:1004B000BC814496A11DB11D8897A105B10518F412
:1004C000C19AC098C29889819A81AB81BC814497B6
:1004D000A109B10986349105A105B10510F4C29AAC
:1004E000C198D601C501865A9F4FAF4FBF4F863482
:1004F0009105A105B10510F4C39AC498D601C501B0
:100500004496A11DB11D8897A105B10518F4C49AA0
:10051000C398C598D601C5014497A109B10986348D
:100520009105A105B10510F4C59AC49880EC0FD2CD
:1005300081E413D280918B0190918C01A0918D0167
:10054000B0918E01B7FF1CC082EC01D28DE205D2C2
:1005500080918B0190918C01A0918D01B0918E01C1
:10056000B095A095909581959F4FAF4FBF4F8093C9
:100570008B0190938C01A0938D01B0938E0104C0E8
:1005800082ECE5D18BE2E9D18091780190917901FB
:10059000A0917A01B0917B01B7FF1CC088ECD7D144
:1005A0008DE2DBD18091780190917901A0917A015F
:1005B000B0917B01B095A095909581959F4FAF4FDD
:1005C000BF4F8093780190937901A0937A01B09303
:1005D0007B0104C088ECBBD18BE2BFD18091830149
:1005E00090918401A0918501B0918601B7FF1CC054
:1005F0008EECADD18DE2B1D18091830190918401D7
:10060000A0918501B0918601B095A09590958195B6
:100610009F4FAF4FBF4F8093830190938401A0936E
:100620008501B093860104C08EEC91D18BE295D107
:1006300083EC8DD180918B0190918C01BCD08AE3A9
:100640008CD189EC84D18091780190917901B3D0DB
:100650008AE383D18FEC7BD18091830190918401D7
:10066000AAD08091920190919301A0919401B091B0
:100670009501B7FF1CC086E96AD18DE26ED18091E9
:10068000920190919301A0919401B0919501B09540
:10069000A095909581959F4FAF4FBF4F809392014A
:1006A00090939301A0939401B093950104C086E9BF
:1006B0004ED18BE252D180917F0190918001A09127
:1006C0008101B0918201B7FF1CC08CE940D18DE25D
:1006D00044D180917F0190918001A0918101B091DE
:1006E0008201B095A095909581959F4FAF4FBF4FD8
:1006F00080937F0190938001A0938101B093820148
:1007000004C08CE924D18BE228D18091870190919B
:100710008801A0918901B0918A01B7FF1CC082EACB
:1007200016D18DE21AD18091870190918801A09114
:100730008901B0918A01B095A095909581959F4FC0
:10074000AF4FBF4F8093870190938801A093890199
:10075000B0938A0104C082EAFAD08BE2FED084E929
:10076000F6D08CE3FAD087E9F2D080919201B2D032
:100770008AE3F3D08DE9EBD080917F01ABD08AE39F
:10078000ECD083EAE4D080918701A4D087EDDFD05C
:1007900088E5E3D08DEDDBD089E5DFD083EED7D0DF
:1007A0008AE5DBD080ED97E0E8ECF0E03197F1F7F7
:1007B0000197D1F7B9CDEF92FF920F931F939C0150
:1007C00068EE73E0C6D6182F092FC90168EE73E0F2
:1007D000C0D6662311F480E302C0862F805DBDD0B1
:1007E000812F902F64E670E0B4D6F82EE92E812F89
:1007F000902F64E670E0ADD6662311F480E302C06A
:10080000862F805DAAD08F2D9E2D6AE070E0A1D644
:10081000362F8F2D9E2D6AE070E09BD6182F332344
:1008200011F480E302C0832F805D97D0812F805D1B
:1008300094D01F910F91FF90EF9008950F931F9305
:100840009C0164E670E085D6182F092FC90164E683
:1008500070E07FD6662311F480E302C0862F805DAE
:100860007CD0812F902F6AE070E073D6362F812FD5
:10087000902F6AE070E06DD6182F332311F480E3D7
:1008800002C0832F805D69D0812F805D66D01F916B
:100890000F9108951F93282F64E64FD6192F822FAA
:1008A0004CD6882311F480E301C0805D56D0812F9F
:1008B0006AE043D6282F812F40D6192F222311F426
:1008C00080E302C0822F805D48D0812F805D45D0BB
:1008D0001F9108951F93282F6AE02FD6382F822F5B
:1008E0002CD6192F332311F480E302C0832F805DAF
:1008F00034D0812F805D31D01F910895805D2DD03F
:1009000008959AE69A95F1F7909892B3807F9F7038
:10091000982B92BB929A85E08A95F1F79298089568
:1009200092B3282F207F9F70292B22BB929A25E01B
:10093000922F9A95F1F7929892B38295807F9F704B
:10094000982B92BB929A2A95F1F7929808959AE67D
:100950009A95F1F79098E4DF08959AE69A95F1F761
:10096000909ADEDF08950F931F9381B3806F81BB50
:10097000889A899A8A9A80E991E028EC30E0F90116
:100980003197F1F70197D9F780E3BBDF80E29EE46E
:100990000197F1F780E3B5DF00EA1FE0C801019796
:1009A000F1F780E3AEDF88E2ACDF88E2D0DF8CE0F5
:1009B000CEDF81E0CCDFC8010197F1F786E0C7DF29
:1009C0001F910F910895CF93DF93EC0102C0219600
:1009D000C4DF88818823D9F7DF91CF910895CF9321
:1009E000DF93EC0104C0FE0184912196B6DF88817B
:1009F0008823C9F7DF91CF9108950F931F93CF9369
:100A0000DF938C01862F90E08770907023E0880F31
:100A1000991F2A95E1F780649ADFC0E0D0E0F801E1
:100A2000EC0FFD1FE4918E2F98DF2196C830D10581
:100A3000B1F7DF91CF911F910F910895A0E0B0E041
:100A4000E3E2F5E09AC5DC012B01FA019C919230BA
:100A500008F439C1EB018881823008F433C1943045
:100A600069F4843009F02FC111969C911197898106
:100A7000981709F428C1ADE6B0E025C1843009F427
:100A800021C18230A9F4923009F01DC19A01AD0153
:100A900088E0EA010990AE01E90109929E018150C6
:100AA000C1F7E201898111969C918923818308C154
:100AB000923009F407C112962D903C901397EB01E8
:100AC0008A819B811496AD90BD90CD90DC90179754
:100AD000EC80FD800E811F819101281B390BB9012B
:100AE00037FF04C066277727621B730B60327105DE
:100AF0000CF061C0121613066CF537014801062E82
:100B000004C096948794779467940A94D2F721E06E
:100B100030E040E050E004C0220F331F441F551F57
:100B20006A95D2F721503040404050402E213F215D
:100B300040235123211531054105510521F021E0C4
:100B400030E040E050E079018A01E628F7280829E2
:100B500019293CC0232BD1F1260E371E3501460141
:100B6000062E04C096948794779467940A94D2F7DB
:100B700021E030E040E050E004C0220F331F441F6A
:100B8000551F6A95D2F721503040404050402A21ED
:100B90003B214C215D21211531054105510521F0F5
:100BA00021E030E040E050E059016A01A628B72872
:100BB000C828D9280BC0821593052CF01C01AA2443
:100BC000BB24650103C0EE24FF24870111969C918C
:100BD000D20111968C91981709F445C0992339F0E8
:100BE000A80197012A193B094C095D0906C0A60115
:100BF00095012E193F09400B510B57FD08C011827A
:100C00003382228224833583468357831DC081E04B
:100C100081833382228288279927DC01821B930BF0
:100C2000A40BB50B84839583A683B7830DC0220FD5
:100C3000331F441F551F2483358346835783828186
:100C400093810197938382832481358146815781E3
:100C5000DA01C9010197A109B1098F5F9F4FAF4F19
:100C6000BF4328F30BC0918333822282EA0CFB1C22
:100C70000C1D1D1DE482F5820683178383E08083AB
:100C8000248135814681578157FF1AC0C901AA279F
:100C900097FDA095BA2F81709070A070B070569596
:100CA000479537952795822B932BA42BB52B8483BF
:100CB0009583A683B78382819381019693838283F0
:100CC000DF0101C0D201CD01CDB7DEB7E2E171C4D1
:100CD000A0E2B0E0EDE6F6E05CC469837A838B8342
:100CE0009C832D833E834F835887E9E0EE2EF12CC1
:100CF000EC0EFD1ECE010196B701A7D38E010F5E4B
:100D00001F4FCE010596B801A0D38A8991E08927AB
:100D10008A8BC701B801AE01475E5F4F8FDEC0D23C
:100D2000A096E6E052C4A0E2B0E0E8E9F6E031C403
:100D300069837A838B839C832D833E834F8358877B
:100D4000F9E0EF2EF12CEC0EFD1ECE010196B7015D
:100D50007CD38E010F5E1F4FCE010596B80175D36F
:100D6000C701B801AE01475E5F4F68DE99D2A09619
:100D7000E6E02BC4A0E2B0E0EFEBF6E0FEC369834F
:100D80007A838B839C832D833E834F835887CE0148
:100D90000196BE01675F7F4F58D3CE010596BE0115
:100DA0006F5E7F4F52D39985923088F08989823067
:100DB000C8F0943019F4823051F404C0843029F41E
:100DC000923081F48DE690E0C6C0923049F420E084
:100DD0009A858A89981321E02A87CE010996BBC09B
:100DE000823049F420E09A858A89981321E02A8B81
:100DF000CE014196B0C02D843E844F8458886D88C2
:100E00007E888F88988CEE24FF248701AA24BB2437
:100E1000650140E050E060E070E0E0E0F0E0C1013A
:100E200081709070892BE9F0E60CF71C081D191DE4
:100E30009A01AB012A0D3B1D4C1D5D1D80E090E029
:100E4000A0E0B0E0E614F7040805190520F481E0FD
:100E500090E0A0E0B0E0BA01A901480F591F6A1F55
:100E60007B1FAA0CBB1CCC1CDD1C97FE08C081E0BC
:100E700090E0A0E0B0E0A82AB92ACA2ADB2A31967D
:100E8000E032F10549F0660C771C881C991C5694D9
:100E9000479437942794C3CFFA85EA892B893C89F4
:100EA0008B859C85280F391F2E5F3F4F17C0CA01C5
:100EB00081709070892B61F016950795F794E794EF
:100EC00080E090E0A0E0B0E8E82AF92A0A2B1B2B8A
:100ED00076956795579547952F5F3F4F77FDE7CFFD
:100EE0000CC0440F551F661F771F17FD4160EE0CA5
:100EF000FF1C001F111F21503040403090E0590767
:100F000090E0690790E4790760F32B8F3C8FDB0159
:100F1000CA018F779070A070B07080349105A105E0
:100F2000B10561F447FD0AC0E114F10401051105A2
:100F300029F0405C5F4F6F4F7F4F40781A8EFE174D
:100F400011F081E08A8F4D8F5E8F6F8F78A383E0E1
:100F5000898FCE014996A4D1A096E2E12AC3A8E1E7
:100F6000B0E0E4EBF7E011C369837A838B839C8361
:100F70002D833E834F835887B9E0EB2EF12CEC0E86
:100F8000FD1ECE010196B70160D28E010F5E1F4F8C
:100F9000CE010596B80159D22985223008F47EC0C9
:100FA0003989323010F4B8017CC08A859A89892742
:100FB0008A87243011F0223031F4231709F06EC0F3
:100FC0006DE670E06EC0343039F41D861E861F86D3
:100FD000188A1C861B8604C0323021F484E089877D
:100FE000B7015FC02B853C858B899C89281B390BF9
:100FF0003C872B87ED84FE840F851889AD88BE88D9
:10100000CF88D88CEA14FB040C051D0540F4EE0CC7
:10101000FF1C001F111F215030403C872B8720E010
:1010200030E040E050E080E090E0A0E0B0E460E03C
:1010300070E0EA14FB040C051D0540F0282B392B49
:101040004A2B5B2BEA18FB080C091D09B695A795DE
:1010500097958795EE0CFF1C001F111F6F5F7F4F48
:101060006F31710531F7DA01C9018F779070A07087
:10107000B07080349105A105B10561F427FD0AC067
:10108000E114F1040105110529F0205C3F4F4F4F99
:101090005F4F20782D873E874F87588BBE01675F53
:1010A0007F4FCB01FDD06896EAE08BC2A8E0B0E0AC
:1010B000EBE5F8E06BC29B01AC0183E08983DA01C8
:1010C000C9018827B7FD83959927AA27BB27B82E82
:1010D000211531054105510519F482E0898339C094
:1010E0008823A9F0203080E0380780E0480780E8B6
:1010F000580729F460E070E080E09FEC2EC0EE24F9
:10110000FF248701E21AF30A040B150B02C07901D0
:101110008A018EE1C82ED12CDC82CB82ED82FE8248
:101120000F831887C801B7016CD0019718161906EC
:1011300084F4082E04C0EE0CFF1C001F111F0A943B
:10114000D2F7ED82FE820F831887C81AD90ADC8293
:10115000CB82BA82CE010196A3D02896E9E032C2B2
:10116000ACE0B0E0E5EBF8E018C269837A838B83EA
:101170009C83CE010196BE016B5F7F4F66D18D814E
:10118000823061F1823050F1843021F48E818823E5
:1011900051F12EC02F81388537FD20C06E812F314F
:1011A00031051CF06623F9F023C08EE190E0821B2C
:1011B000930B29853A854B855C8504C056954795E8
:1011C000379527958A95D2F76623B1F050954095CB
:1011D000309521953F4F4F4F5F4F0EC020E030E0DC
:1011E00040E050E009C02FEF3FEF4FEF5FE704C052
:1011F00020E030E040E050E8B901CA012C96E2E07E
:10120000E8C1EF92FF920F931F937B018C0180E066
:10121000E81680E0F80681E0080780E0180788F407
:101220008FEFE816F1040105110531F028F088E090
:1012300090E0A0E0B0E017C080E090E0A0E0B0E077
:1012400012C080E0E81680E0F80680E0080781E040
:10125000180728F088E190E0A0E0B0E004C080E149
:1012600090E0A0E0B0E020E230E040E050E0281B59
:10127000390B4A0B5B0B04C016950795F794E7945E
:101280008A95D2F7F701EB58FF4F8081281B31096F
:1012900041095109C9011F910F91FF90EF900895E5
:1012A000DF92EF92FF920F931F93FC01E480F58091
:1012B00006811781D1808081823048F480E090E0FF
:1012C000A0E1B0E0E82AF92A0A2B1B2BA5C0843044
:1012D00009F49FC0823021F4EE24FF24870105C069
:1012E000E114F1040105110519F4E0E0F0E096C005
:1012F000628173819FEF623879070CF05BC022E84E
:101300003FEF261B370B2A3131052CF020E030E06F
:1013100040E050E02AC0B801A701022E04C0769533
:101320006795579547950A94D2F781E090E0A0E041
:10133000B0E004C0880F991FAA1FBB1F2A95D2F7DF
:101340000197A109B1098E219F21A023B123009704
:10135000A105B10521F081E090E0A0E0B0E09A01A4
:10136000AB01282B392B4A2B5B2BDA01C9018F7774
:101370009070A070B07080349105A105B10539F46A
:1013800027FF09C0205C3F4F4F4F5F4F04C0215CD7
:101390003F4F4F4F5F4FE0E0F0E02030A0E03A07D2
:1013A000A0E04A07A0E45A0710F0E1E0F0E079017C
:1013B0008A0127C06038710564F5FB01E158FF4FD1
:1013C000D801C7018F779070A070B07080349105FC
:1013D000A105B10539F4E7FE0DC080E490E0A0E07E
:1013E000B0E004C08FE390E0A0E0B0E0E80EF91EAA
:1013F0000A1F1B1F17FF05C016950795F794E79462
:10140000319687E016950795F794E7948A95D1F77A
:1014100005C0EE24FF248701EFEFF0E06E2F679503
:1014200066276795902F9F77D794DD24D7948E2FCA
:101430008695492F462B582F5D29B701CA011F9168
:101440000F91FF90EF90DF900895FC01DB01408148
:1014500051812281622F6F7770E0221F2227221F85
:101460009381892F880F822B282F30E0991F99278D
:10147000991F11969C93119721153105A9F54115D6
:1014800051056105710511F482E037C082E89FEFD4
:1014900013969C938E9312979A01AB0167E0220FEB
:1014A000331F441F551F6A95D1F783E08C930DC0FD
:1014B000220F331F441F551F12968D919C91139735
:1014C000019713969C938E931297203080E03807F3
:1014D00080E0480780E4580758F314962D933D9315
:1014E0004D935C93179708952F3F310579F441157B
:1014F00051056105710519F484E08C93089564FF2A
:1015000003C081E08C9312C01C9210C02F57304052
:1015100013963C932E93129783E08C9387E0440FAD
:10152000551F661F771F8A95D1F7706414964D93E7
:101530005D936D937C9317970895991B79E004C090
:10154000991F961708F0961B881F7A95C9F7809502
:101550000895AA1BBB1B51E107C0AA1FBB1FA617FA
:10156000B70710F0A61BB70B881F991F5A95A9F74C
:1015700080959095BC01CD0108952F923F924F9296
:101580005F926F927F928F929F92AF92BF92CF9213
:10159000DF92EF92FF920F931F93CF93DF93CDB71C
:1015A000DEB7CA1BDB0B0FB6F894DEBF0FBECDBF94
:1015B00009942A88398848885F846E847D848C8465
:1015C0009B84AA84B984C884DF80EE80FD800C816E
:1015D0001B81AA81B981CE0FD11D0FB6F894DEBF51
:1015E0000FBECDBFED010895DF93DD27B92FBF7783
:1015F00040E85FE31616170648075B0710F4D92F7B
:1016000051D09F938F937F936F93F6D0E6E2F0E0F3
:1016100013D037D02F913F914F915F9154D0DD235C
:1016200049F09058A2EA2AED3FE049EC5FE3D07818
:101630005D27F2D0DF9125C0DF93CF931F930F93E7
:10164000FF92EF92DF927B018C01689405C0DA2E45
:10165000EF0139D0FE01E894A5912591359145918E
:101660005591AEF3EF01D8D0FE019701A801DA94AD
:1016700079F7DF90EF90FF900F911F91CF91DF915D
:101680000895092E0394000C11F4882352F0BB0F27
:1016900040F4BF2B11F460FF04C06F5F7F4F8F4F8A
:1016A0009F4F08959B01AC0160E070E080E89FE3EC
:1016B00056CC23D128F028D118F0952309F0FFC08B
:1016C00012C111244BC127D1A0F3959FD1F3950FDF
:1016D00050E0551F629FF001729FBB27F00DB11DB6
:1016E000639FAA27F00DB11DAA1F649F6627B00D46
:1016F000A11D661F829F2227B00DA11D621F739F2F
:10170000B00DA11D621F839FA00D611D221F749F3C
:101710003327A00D611D231F849F600D211D822F83
:10172000762F6A2F11249F5750408AF0E1F08823CA
:101730004AF0EE0FFF1FBB1F661F771F881F9150D7
:101740005040A9F79E3F510570F0B9C007C15F3FF7
:10175000ECF3983EDCF3869577956795B795F7950A
:10176000E7959F5FC1F7FE2B880F911D9695879592
:1017700097F9089511F40EF4B6C0A7C0D4D0D0F3F1
:101780009923D9F3CEF39F57550B87FFAFD0002491
:10179000A0E640EA900180585695979528F4805C21
:1017A000660F771F881F20F026173707480730F489
:1017B000621B730B840B202931294A2BA6951794A1
:1017C0000794202531254A2758F7660F771F881F71
:1017D00020F026173707480730F4620B730B840B91
:1017E000200D311D411DA09581F7B901842F91581D
:1017F000880F9695879508959B01AC01BBCA7DD053
:1018000030F082D020F031F49F3F11F41EF46BC011
:101810000EF4E095E7FB53C0E92F7DD080F3BA17B3
:10182000620773078407950718F071F49EF595C059
:101830000EF4E0950B2EBA2FA02D0B01B9019001EB
:101840000C01CA01A0011124FF27591B99F0593F2F
:1018500050F4503E68F11A16F040A22F232F342F77
:101860004427585FF3CF469537952795A795F040C5
:101870005395C9F77EF41F16BA0B620B730B840BDA
:10188000BAF09150A1F0FF0FBB1F661F771F881F92
:10189000C2F70EC0BA0F621F731F841F48F48795EA
:1018A00077956795B795F7959E3F08F0B3CF9395D9
:1018B000880F08F09927EE0F97958795089597F967
:1018C0009F6780E870E060E008959F3F31F091509D
:1018D00020F4879577956795B795880F911D969514
:1018E000879597F908959FEF80EC089591505040A7
:1018F000660F771F881FD2F7089500240A941616E2
:10190000170618060906089500240A9412161306ED
:1019100014060506089557FD9058440F551F59F0B9
:101920005F3F71F04795880F97FB991F61F09F3FCC
:1019300079F087950895121613061406551FF2CFF5
:101940004695F1DF08C0161617061806991FF1CF45
:1019500086957105610508940895E894BB2766276C
:0C1960007727CB0197F90895F894FFCF8A
:10196C004144584C333435207465737400000000C6
:10197C00000000000000010202030303030404043E
:10198C000404040404050505050505050505050500
:10199C0005050505050606060606060606060606E0
:1019AC0006060606060606060606060606060606CB
:1019BC0006060606060707070707070707070707B0
:1019CC00070707070707070707070707070707079B
:1019DC00070707070707070707070707070707078B
:1019EC00070707070707070707070707070707077B
:1019FC000707070707080808080808080808080860
:101A0C00080808080808080808080808080808084A
:101A1C00080808080808080808080808080808083A
:101A2C00080808080808080808080808080808082A
:101A3C00080808080808080808080808080808081A
:101A4C00080808080808080808080808080808080A
:101A5C0008080808080808080808080808080808FA
:101A6C0008080808080808080808080808080808EA
:061A7C000808080808003C
:00000001FF
